:0200000480007A
:10000000130000001300000013000000971104000B
:100010009381C1C1170106001301C1FE171500002D
:1000200013054574970504009385C5FD1706040064
:100030001306C63F63FCC5008322050023A05500BC
:100040001305450093854500E3E8C5FE1705040048
:100050001305C53D970504009385453D6378B500BC
:100060002320050013054500E36CB5FE9700000052
:10007000130101FF23241100371500001305058823
:100080007310453037250000130585807310053047
:100090001305000093050000EF00C0126F104035FB
:1000A0006F000000130000001300000013000000A8
:1000B000130101F8232211002324210023263100FB
:1000C00023284100232A5100232C6100232E710094
:1000D00023208102232291022324A1022326B1029C
:1000E0002328C102232AD102232CE102232EF1026C
:1000F0002320010523221105232421052326310570
:1001000023284105232A5105232C6105232E71053F
:1001100023208107232291072324A1072326B10747
:100120002328C107232AD107232CE107232EF10717
:10013000EF00800883204100032181008321C1005A
:100140000322010183224101032381018323C10191
:100150000324010283244102032581028325C10275
:100160000326010383264103032781038327C10359
:100170000328010483284104032981048329C1043D
:10018000032A0105832A4105032B8105832BC10521
:10019000032C0106832C4106032D8106832DC10605
:1001A000032E0107832E4107032F8107832FC107E9
:1001B00013010108730020306F00000000000000F0
:0401C000000000003B
:1001C400130101FE232C8100171500001305C555EA
:1001D40037240000232A91002328210123263101FA
:1001E400232E110013040471EF00107D97190000F1
:1001F40093898954B70403F0171900001309C954EB
:100204009305040013850900EF00107B23A08400EC
:1002140083A504001305090013041400EF00D0792A
:100224006FF01FFE97070080938787DD99C7171526
:1002340000001305052A6F10202D82806376D600F6
:10024400B385C5002380A500678000006780000097
:10025400130101FD0323810323202103232E3101F4
:10026400232C4101232A51012328610123267101F2
:1002740023248101232611022324810223229102B3
:10028400232291012320A101137C2300138B060058
:10029400130A0500938A0500930906001309070051
:1002A40083260103832B410363140C061375130087
:1002B400639A0B1C63F6D7021307F0016364F732E9
:1002C40013060003930500026F008000638AB700E1
:1002D400938717003307F900A30FC7FEE3E8D7FE9F
:1002E4006308050263F6770313070002638EE71AB7
:1002F40013060003930500026F0080006386B71A9B
:10030400938717003307F900A30FC7FEE39877FF1D
:100314001377030163020708137703406314071A72
:10032400639E0718130700016382E82A93072000DD
:10033400638EF826930700032300F9009307100047
:100344006304081A3307F900138417009307D002D3
:100354002300F7001373330063140300636A740FFC
:10036400938C09006F00C00413070002638AE7023C
:10037400B306F90093871700130780072380E6006C
:1003840013070002638EE7003307F90093060003A6
:100394002300D7009387170013070002E392E7FABC
:1003A400137333006302030A938C090013040002DD
:1003B400B38C8C00330D9901330489000345F4FF99
:1003C40033068D4093060B001304F4FF93850A0053
:1003D40093840C00E7000A00E31289FE63080C0210
:1003E400B389344163F479031386040093060B0044
:1003F40093850A001305000293841400E7000A00A1
:100404009389190013860400E3E279FF8320C10273
:100414000324810213850400032901028324410279
:100424008329C101032A8101832A4101032B01018C
:10043400832BC100032C8100832C4100032D010078
:10044400130101036780000013040002637C740B32
:10045400B38C7901B38C8C401386090093060B008E
:1004640093850A001305000293041600E7000A00AE
:1004740013860400E39494FF93840C00E31A04F2BB
:100484006FF0DFF5630E05086316080A1377C300DF
:100494006312070AE3F8D7E41307F001E372F7E203
:1004A40093070002E3F677E793770301E38A07EE05
:1004B400937703406390070E930700026380F60866
:1004C400638E770713070001638AE8081307200087
:1004D400E398E8EA13070002E384E7EC3307F90042
:1004E400938717006F00C00D137743006310070252
:1004F400137783006316070813733300138407000C
:10050400E30603F4938C09006FF01FF73307F90037
:10051400138417009307B0022300F7006FF09FE3E2
:10052400E3F8D7DE1307F001E37CF7D89307000262
:100534006FF01FDE938BFBFF6FF0DFF51387F7FF80
:10054400630E0704930600016380D80C9306200011
:100554006386D806930707006FF01FE3137703023F
:10056400E30407E013070002E38CE7E23307F90032
:10057400930680052300D700938717006FF05FE090
:100584003307F90013841700930700022300F700D0
:100594006FF05FDC930700026FF0DFF29307000156
:1005A4006388F80493072000E396F8FA930720067B
:1005B4002300F900930710006FF01FDD3307E900F3
:1005C400930620062300D7006FF09FDB1377030206
:1005D400E31E07F8930780072300F9009307100030
:1005E4006FF09FDA93070002E31E05CE6FF05FD22F
:1005F40093770302E38007FE930780052300F90045
:10060400930710006FF05FD8937603029387E7FF98
:10061400E39E06F4B306F900930707006FF0DFD5F5
:10062400130101FB232E3103232611042324810407
:10063400232291042320210583294105631A0704F9
:1006440013F309409300010193F9F9FE63020304D3
:1006540003230105232431012320110123226100F6
:100664009308080013880700930707001387000006
:10067400EFF01FBE8320C1040324810483244104BA
:10068400032901048329C1031301010567800000C4
:1006940013FE090213031006631C0E081379F30FEB
:1006A400930F07001353F701930001011307000090
:1006B400930310009302F0FF13049000130969FFE1
:1006C40093040002130F0000130EE001B3DECF41C8
:1006D40093FE1E001313130033E36E00B39EC30195
:1006E400130EFEFF6346030133030341336FDF013F
:1006F400E31E5EFC1373F30F6366640213030303C8
:100704001373F30F13071700338EE000A30F6EFE6D
:10071400E3000FF4E30E97F213030000930F0F00AE
:100724006FF05FFA330323011373F30F6FF09FFD30
:10073400130310046FF09FF6130101F7232C8106B5
:1007440023206107232E71052328A1052326B10543
:10075400232E1106232A9106232821072326310755
:100764002324410723225107232C8105232A9105A1
:10077400232611093363F700232CA100232EB10093
:10078400130B0600938B0600130D08001384080056
:10079400832E0109832DC1096316030893F60D40C6
:1007A40093FDFDFE6380060893090000130A01020D
:1007B400832781098325C101032581012322F100B7
:1007C400832741092324B101930804002320F10065
:1007D40013080D009387090013070A0093860B0082
:1007E40013060B00EFF0DFA68320C1070324810763
:1007F40083244107032901078329C106032A8106AB
:10080400832A4106032B0106832BC105032C810592
:10081400832C4105032D0105832DC1041301010916
:100824006780000013F60D0293061006631E060E81
:100834009384070093D5F40193070700130E000077
:1008440093090000130A01029300F0011309100038
:100854009308F0FF930A9000938C66FF130C000238
:100864001307E003130F000013030000939F140009
:100874003386E04093D2F50193161E0033D5E7008A
:100884003396CF00130807FEB3E6D2009395150004
:100894003365A6006344080033D50441137515007D
:1008A400B365B500138E060063C8D6033316E9009A
:1008B40033858540B3B2A500B383D6411358F641BE
:1008C4006394DE0063EA850093050500338E53408C
:1008D400336FCF00336303011307F7FFE31A17F9EC
:1008E40093F5F50F63ECBA029385050393F7F50FBF
:1008F4009389190033073A01A30FF7FEB3676F001A
:10090400E38807EAE38689EB9355F301130E0000AD
:1009140093070F00930403006FF09FF4B3859501D0
:1009240093F7F50F6FF0DFFC930610046FF05FF0A0
:10093400130101FA23282105232631052324410527
:10094400232C81032326B103232E1104232C810499
:10095400232A91042322510523206105232E7103A8
:10096400232A91032328A103938905001309060070
:10097400138C0600930D0700170A0000130A4A8D12
:1009840063840500130A050003450C00130D0000E1
:1009940063040516B70701009387F7FF930400016A
:1009A400971C0000938C0CBF130B9000232AF100BA
:1009B4006F00000213060D009306090093850900D9
:1009C400130D1D00E7000A0003450C006306051221
:1009D40093075002130C1C00E31EF5FC03450C00A6
:1009E40013071C0093060000930705FE93F7F70F07
:1009F4001306070063ECF40293972700B38797016B
:100A040083A70700B38797016780070093E6160062
:100A1400130C070003450C0013071C001306070002
:100A2400930705FE93F7F70FE3F8F4FC930705FD2E
:100A340093F7F70F6370FB129307A0026308F51C8A
:100A44009307E00213060C00930B0000130C07003D
:100A5400930F00006304F5149307A0066306F516CC
:100A640063FEA7069307C006630AF53C9307A00735
:100A74006318F5000345160093E60610130C1C00DA
:100A84009307B5FD93F7F70F13073005E364F7F207
:100A940017170000130747B493972700B387E7009D
:100AA40083A70700B387E7006780070093E6260063
:100AB400130C07006FF01FF693E64600130C0700B3
:100AC4006FF05FF593E60601130C07006FF09FF4D7
:100AD40093E68600130C07006FF0DFF3930780069C
:100AE400E310F5FA03451600630EF53893E606089D
:100AF400130C1C006FF0DFF813060D0063642D0166
:100B04001306F9FF930609009385090013050000F5
:100B1400E7000A008320C1050324810513050D00A5
:100B240083244105032901058329C104032A81047F
:100B3400832A4104032B0104832BC103032C810367
:100B4400832C4103032D0103832DC10213010106EC
:100B540067800000930B00006F00C000130C0700B7
:100B64001307170013942B00330474011314140097
:100B74003304A4000345070013060700930B04FD88
:100B8400930705FD93F7F70FE37AFBFC130C2C0096
:100B94009307E002930F0000E310F5EC0345160001
:100BA40093E60640930705FD93F7F70F6378FB027E
:100BB4009307A0026300F52A9307A00613060C000E
:100BC400130C1C00E31EF5E893E60620034516000B
:100BD400130C1C006FF0DFEA130C0600939A2F002D
:100BE400B38AFA01939A1A00B38AAA0003451C0037
:100BF40013061C00938F0AFD930705FD93F7F70F67
:100C0400E37CFBFC130C2C006FF01FE583AB0D00A1
:100C1400938D4D0063CC0B2003451C00130C2C005A
:100C24006FF01FF703A40D0093874D00232CF100F0
:100C34000345040063920F24930DE0FF630A0552F9
:100C440093871D002328F1003306F4009307040062
:100C54006F008000638CC7009387170003C70700E9
:100C6400E31A07FEB38787402328F10093FA06406E
:100C740063880A008327010163F4FF002328F1013C
:100C840093F72600232EF100638407366308052CAE
:100C9400638C0A28B38AAF0113060D006386CA0267
:100CA4009306090093850900930D1600E7000A00D6
:100CB400B387AD41B307F40003C50700630C052CEB
:100CC40013860D00E39ECAFC8327C101138D0A001D
:100CD40063960728832D81016FF01FCF03A70D00B2
:100CE40013E41602930780002320F10013060D007D
:100CF4002322810093880F0013080001930700004A
:100D0400930609009385090013050A00EFF05F912B
:100D1400938D4D00130D05006FF01FCB93874D008D
:100D2400930A1D0093F626002328F10013840A0079
:100D34006386062603C50D0013060D0093060900FD
:100D440093850900E7000A0013071000338DAB01F7
:100D54006378773B93071400130604009306090095
:100D6400138407009385090013050002E7000A00B5
:100D7400E3128DFE832D01016FF01FC593078007D9
:100D84006304F53C930780056306F5109307F006AA
:100D94006302F53293072006630AF51013079006E1
:100DA40013F6F6FE93F706401308A0006314E5104B
:100DB40013F40620638A07101376E6FF9307900660
:100DC400137406206302F51093074006630EF50EB4
:100DD4006318042E9377061013844D00639A073426
:100DE40093770604639A07309377060803A70D00E8
:100DF40063860700832741013377F7002322C1006C
:100E04002320710193880F00930700006F00C00F27
:100E140013060D009306090093850900130550027B
:100E2400130D1D00E7000A006FF01FBA93E62600B9
:100E3400B30B704103451C006FF05FDE03451600E1
:100E4400E31CF5C293E6063003452600130C360076
:100E54006FF01FC383AF0D0003452600130C36004B
:100E640093C7FFFF93D7F741B3FFFF00938D4D0066
:100E7400130626006FF05FBE630C052E938DFFFFF3
:100E84006FF01FDC93E6060C03452600130C3600B6
:100E94006FF01FBF13F636FF93F706401366060282
:100EA40063840720130800016FF01FF1130820006A
:100EB400138606001307400693770640631AE52C51
:100EC40013740620E39A07EE631E04169377061044
:100ED40013844D00639C07229377060463980720CC
:100EE40093770608638C072683970D0093D6F74102
:100EF40033C7F6003307D7402322C10023207101F2
:100F040093880F0093D7F70113060D009306090089
:100F14009385090013050A00EFF08FF0130D050007
:100F2400930D04006FF05FAA13060D0093060900E9
:100F340093850900930A1600E7000A00B387AA41C3
:100F4400B307F40003C5070013860A00E31005FE87
:100F5400138D0A008327C101E38E07D6832701017D
:100F640013060D00E3F877D73384AB01330DF44057
:100F74009306090093850900130500021304160063
:100F8400E7000A0013060400E314A4FF832D810183
:100F94006FF09FA3138D0D006FF0DFFB130710009C
:100FA4006372771F1304FDFF330474016F00800024
:100FB400938A1A0013060D0093060900938509000D
:100FC40013050002138D0A00E7000A00E3928AFE6B
:100FD400138D1A0003C50D009306090013060400BF
:100FE40093850900E7000A00832D01016FF0DF9D5E
:100FF400032701019307170063707719B387AB01C7
:10100400B38DE7402328F10193071D0013060D005B
:10101400930609009385090013050002138D070048
:10102400E7000A00832F0101E31EBDFD0345040010
:1010340093871B002328F100E31C05C4832D810141
:101044006FF09F98938D7D0093FD8DFF03A54D0058
:1010540083A70D00930808009356F541B3C7F60023
:101064003387D740B3C5A600B3B7E700B386D540EE
:101074002326C100232471012322F101232001002E
:101084001358F501B387F64013060D0093060900C3
:101094009385090013050A00EFF00FEA938D8D0084
:1010A400130D05006FF05F9213F40620130800017E
:1010B4006FF01FD213088000138606006FF09FDFC5
:1010C400938D7D0093FD8DFF03A70D0083A74D0035
:1010D400930808002326C100232471012322F1016F
:1010E40023200100130800006FF01FFA83C70D00CE
:1010F400138707006FF05FE003C70D006FF01FD088
:10110400138D0A00832D01016FF01F8C83A70D003E
:1011140093880F002322C10013D7F741B346F70089
:101124002320710193D7F7013387E6406FF0DFDDA9
:1011340003A70D0093880F002322C100232071010F
:10114400930700006FF05FDC93F70640130800017B
:1011540013F636FFE38407C66FF01FC683A70D009E
:1011640093D6F74133C7F6003307D7406FF0DFD883
:10117400232801006FF09FAF2328F100E31A05B084
:101184006FF0DFEB13040D00138D0A006FF09FE482
:10119400930606006FF0DFFB631405006780000010
:1011A4006F00801A6308050003A3050083A54500AA
:1011B4006700030067800000130101FC1303410270
:1011C4002322B1022324C1022326D1022328E102CF
:1011D4009306050093058100130703001306F0FF2F
:1011E40017050000130585FB232E1100232AF102A5
:1011F400232C0103232E110323266100EFF04FF368
:101204008320C1011301010467800000130101FC64
:10121400130381022324C1022326D1022328E102DD
:101224009386050013070300930505001306F0FFDA
:1012340017F5FFFF1305C500232E1100232AF10221
:10124400232C0103232E110323266100EFF04FEE1C
:101254008320C1011301010467800000130101FC14
:101264001303C1022326D1022328E10293060600B8
:1012740013070300138605009305050017F5FFFF08
:10128400130505FC232E1100232AF102232C01034C
:10129400232E110323266100EFF08FE98320C1017F
:1012A4001301010467800000130101FE1387050088
:1012B400930605009305C1001306F0FF170500000F
:1012C4001305C5ED232E1100EFF08FE68320C10135
:1012D40013010102678000001387060093060600CD
:1012E400138605009305050017F5FFFF130545F563
:1012F4006FF00FE4130101FC1303C1022326D10292
:101304002328E1022324A1002326B100930606002A
:1013140093058100130703001306F0FF170500006F
:10132400130585E8232E1100232AF102232C01033F
:10133400232E110323226100EFF08FDF8320C101EC
:101344001301010467800000130101FEA307A1003B
:10135400930510001305F100232E1100EF00C001C6
:101364008320C10113010102678000001385050079
:10137400930506006F004000638605023306B5003E
:10138400370701F0834605008327470093D70701F9
:1013940093F7F70FE38A07FE2320D7001305150000
:1013A400E312A6FE678000008346050063840602FC
:1013B400370701F08327470093D7070193F7F70F07
:1013C400E38A07FE2320D700130515008346050092
:1013D400E39206FE67800000F32500B8732500B091
:1013E400732600B8E39AC5FE678000004111814569
:1013F40022C406C62A841928970700009387C73594
:1014040088435C5D91C3829722854922797197074D
:1014140000009387673462C403AC07004ECE52CCFD
:1014240056CA5AC806D622D426D24AD05EC6AA8A3A
:101434002E8B054AFD5903298C1463040902832465
:1014440049001384F4FF634E04008A04CA946306BB
:101454000B0283A74410638267037D14F114E3181D
:1014640034FFB250225492540259F249624AD24A89
:10147400424BB24B224C4561828083274900D440C1
:10148400FD176380870423A20400E1DA8327891807
:1014940033178A00832B4900F98F99EB82968327AF
:1014A4004900E39A77F983278C14E38827FB61B713
:1014B4008327C91883A544087D8F19E7568582962A
:1014C400F9BF23228900D1B72E858296C9BF411165
:1014D40022C4970700009387A72817040000130469
:1014E40024281D8C06C626C2098411C8931424001E
:1014F400F114BE949C407D14F114829765FCB240B3
:101504002244924441018280AA85814601460145D4
:1015140009A09707000093872724984383278714FB
:10152400A1C3D8437D48634DE804131827001DC1A7
:10153400338307012324C30883A887180546331679
:10154400E600B3E8C80023A417192324D31089465E
:10155400630DD5000507D8C3C2978CC701458280A7
:101564009307C7142324F7146DBF83A6C718050770
:10157400D8C3558E23A6C718C2978CC7014582804D
:101584007D55828067800000678000006F00000046
:1015940040F5FFFF9CF4FFFF9CF4FFFF34F5FFFFD1
:1015A4009CF4FFFF9CF4FFFF9CF4FFFF9CF4FFFFFF
:1015B4009CF4FFFF9CF4FFFF9CF4FFFF28F5FFFF62
:1015C4009CF4FFFF1CF5FFFF9CF4FFFF9CF4FFFF5E
:1015D4007CF4FFFF3CF8FFFFE0F3FFFFE0F3FFFFC5
:1015E400E0F3FFFFE0F3FFFFE0F3FFFFE0F3FFFFB3
:1015F400E0F3FFFFE0F3FFFFE0F3FFFFE0F3FFFFA3
:10160400E0F3FFFFE0F3FFFFE0F3FFFFE0F3FFFF92
:10161400E0F3FFFFE0F3FFFFE0F3FFFFE0F3FFFF82
:10162400E0F3FFFFE0F3FFFFE0F3FFFFE0F3FFFF72
:10163400E0F3FFFFE0F3FFFFE0F3FFFFE0F3FFFF62
:10164400E0F3FFFFE0F3FFFFE0F3FFFFE0F3FFFF52
:10165400E0F3FFFFE0F3FFFFE0F3FFFFE0F3FFFF42
:10166400E0F3FFFFE0F3FFFFE0F3FFFFE0F3FFFF32
:10167400E0F3FFFFE0F3FFFFE0F3FFFFE0F3FFFF22
:10168400E0F3FFFFE0F3FFFFE0F3FFFFE0F3FFFF12
:10169400E0F3FFFFE0F3FFFFE0F3FFFFE0F3FFFF02
:1016A400A8F7FFFFE0F3FFFFE0F3FFFFE0F3FFFF26
:1016B400E0F3FFFFE0F3FFFFE0F3FFFFE0F3FFFFE2
:1016C400E0F3FFFFE0F3FFFFA8F7FFFF48F7FFFF9A
:1016D400A8F7FFFFE0F3FFFFE0F3FFFFE0F3FFFFF6
:1016E400E0F3FFFFA8F7FFFFE0F3FFFFE0F3FFFFE6
:1016F400E0F3FFFFE0F3FFFFE0F3FFFFA8F7FFFFD6
:1017040008F7FFFFE0F3FFFFE0F3FFFF50F6FFFFF2
:10171400E0F3FFFFA8F7FFFFE0F3FFFFE0F3FFFFB5
:10172400A8F7FFFF48454C4C4F20574F524C440AF2
:1017340000000000537461746520696E203A20250E
:10174400690A00005374617465206F75743A20252A
:08175400690A00000000048096
:04175C0028020080DF
:1017600000000000EC02048054030480BC030480E9
:101770000000000000000000000000000000000069
:101780000000000000000000000000000000000059
:101790000000000000000000000000000000000049
:1017A0000000000000000000000000000000000039
:1017B0000000000000000000000000000000000029
:1017C0000000000000000000000000000000000019
:1017D0000000000000000000000000000000000009
:1017E00000000000000000000000000000000000F9
:1017F00000000000000000000000000000000000E9
:1018000000000000000000000100000000000000D7
:101810000E33CDAB34126DE6ECDE05000B0000009C
:1018200000000000000000000000000000000000B8
:1018300000000000000000000000000000000000A8
:101840000000000000000000000000000000000098
:101850000000000000000000000000000000000088
:040000058000000077
:00000001FF
